:100000000C9448000C9465000C9465000C946500F9
:100010000C9465000C9465000C9465000C946500CC
:100020000C9465000C94B7000C9465000C9465006A
:100030000C9465000C9465000C9465000C946500AC
:100040000C9465000C9428030C94F3010C94AF01FC
:100050000C949A010C9465000C9465000C94650056
:100060000C9465000C9465006374726C5F616C6C39
:100070006F6328256429206964783D25640A007E21
:100080000E0E0E0E1B1B1C0E1B1B7E0E0E0E0E00EC
:1000900011241FBECFEFD4E0DEBFCDBF11E0A0E042
:1000A000B1E0EAE0FAE202C005900D92A231B10798
:1000B000D9F712E0A2E1B1E001C01D92A43AB10764
:1000C000E1F70E9470000C9403150C9400008091DD
:1000D00012010895A8950E947C030E949F10089524
:1000E000F894A8950E9450010E94EE020E94730F9E
:1000F0008FEF80931001409A0E947601789480E0FF
:1001000090E060E040E050E00E94FF1080E090E06E
:100110000E94AA0F0E945A0D0E9494020E948E080B
:100120000E946A00F9CF909112019817F1F0963071
:10013000E1F0953011F48630C1F4809312010E94F1
:10014000DD0480911201853029F480E060E245E011
:100150000E94A61180911201863029F480E060E2AD
:1001600046E00E94A61181E0089580E008951F9264
:100170000F920FB60F9211248F939F93AF93BF935B
:1001800080919A02882329F080919A02815080936D
:100190009A0280911301882329F581E0809313014D
:1001A0007894809114018F5F8093140180911401E1
:1001B00090E083709070892B99F4809196029091D1
:1001C0009702A0919802B09199020196A11DB11DCC
:1001D0008093960290939702A0939802B09399020D
:1001E00010921301BF91AF919F918F910F900FBE0D
:1001F0000F901F90189510929602109297021092ED
:10020000980210929902E0E7F0E010821092B0009C
:1002100082E08093B1008081816080830895EF92B5
:10022000FF920F931F932091960230919702409175
:100230009802509199027C0100E010E0E20EF31E5A
:10024000041F151F02C00E946A00C801B7010E9466
:10025000C1118823C1F31F910F91FF90EF90089572
:10026000EF92FF920F931F93209196023091970285
:1002700040919802509199027C0100E010E0E20E5A
:10028000F31E041F151F01C0A895C801B7010E94E5
:10029000C1118823C9F31F910F91FF90EF9008952A
:1002A000EAEFFFE39491892F81508E3F10F49093F1
:1002B00066000895ECEFFFE3259135914591549147
:1002C0005070B901CA010895EFEFFFE3E4918E2F5A
:1002D0000895F8942CE088E190E00FB6F894A89582
:1002E000809360000FBE20936000FFCF1092160134
:1002F00080911601E6E1F1E08293808180933001E4
:100300008091300180932F01519A5098599A589AB0
:100310005A9882E08093C0001092C5008FE08093CD
:10032000C40086E08093C2008CEF8093C10080E01F
:1003300090E008951F920F920FB60F9211248F93A1
:100340001092160180911601809315015A988091A0
:10035000C6008F910F900FBE0F901F9018951F929F
:100360000F920FB60F9211248F939F93EF93FF93E9
:1003700090912F0180913001981731F48091C10044
:100380008F7D8093C10026C05A9A8091390187FFE2
:1003900009C0809139018F77809339018091C10024
:1003A000816003C08091C1008E7F8093C100E09185
:1003B0003001F0E0EB5EFE4F848D8093C6008091AB
:1003C00030018F5F8093300180913001883010F0D0
:1003D00010923001FF91EF919F918F910F900FBE7E
:1003E0000F901F9018951F920F920FB60F92112425
:1003F0002F933F938F939F93EF93FF935A9B03C049
:100400008091C60030C0209115018091160130E026
:1004100090E001972817390741F080911501873145
:1004200079F480911601882359F4809116018F5F29
:100430008093160180911601883110F010921601F8
:10044000E0911501F0E08091C600EB5EFE4F8283E3
:10045000809115018F5F809315018091150188317E
:1004600010F010921501FF91EF919F918F913F91A4
:100470002F910F900FBE0F901F901895482FA895A1
:1004800007C08091C10080628093C1007894A895D4
:1004900020912F018091300130E090E001972817E2
:1004A000390779F380912F01873021F48091300151
:1004B000882339F3E0912F01F0E0EB5EFE4F448F8B
:1004C00080912F018F5F80932F0180912F018830C1
:1004D00010F010922F018091C10080628093C100C2
:1004E000842F0895282F5A99FECF80913901806872
:1004F00080933901109216018091160180931501A5
:100500002F77A22FA295AF70B0E0A050BF4FE22F7F
:10051000F0E0EF70F070E050FF4F8C9190818927F0
:10052000822B0E943E0208955A991CC09091150199
:10053000809116019817B1F0E0911601F0E0EB5EA2
:10054000FE4F9281F894809116018F5F809316017F
:1005500080911601883110F010921601292F30E099
:10056000789402C02FEF3FEFC90108958BB190E05E
:10057000969587959695879581700895EF92FF924D
:100580000F931F939C01181619061CF58091960273
:1005900090919702A0919802B09199027901002759
:1005A000F7FC0095102FE80EF91E0A1F1B1F809103
:1005B000C100877F8093C1005A9A599A02C00E9455
:1005C0006A00C801B7010E94C1118823C1F30E94CB
:1005D00076011F910F91FF90EF9008951092C10046
:1005E0001DBA10926800EDE6F0E010828081ECE622
:1005F000F0E08083808180936B0093E09CBB87E078
:100600008BBB1CBC94B915B881E087B98EE388B95F
:100610008EEF8AB99BB90E94FB00A8952EE088E175
:1006200090E00FB6F894A895809360000FBE2093D9
:100630006000089584B1837C84B985B1837C85B9D9
:1006400084EE8CBD01C08EB50DB407FCFCCF0895BF
:100650001F920F920FB60F9211242F933F934F9337
:100660005F936F937F938F939F93AF93BF93EF931A
:10067000FF9380919B0290919C022FEF8F3F9207F6
:1006800079F0249A8EBD0DB406FE03C024980E9412
:10069000FC0D8FEF9FEF90939C0280939B0201C013
:1006A00024988EB50E94780E8DB59EB587FDFCCF3F
:1006B00086FDFACFFF91EF91BF91AF919F918F91FE
:1006C0007F916F915F914F913F912F910F900FBE4E
:1006D0000F901F9018958091960290919702A0918B
:1006E0009802B091990280933A0190933B01A093B4
:1006F0003C01B0933D010895809110018F3F09F1B5
:1007000060913A0170913B0180913C0190913D01D3
:100710006115710581059105B1F06C507E4F8F4FC9
:100720009F4F0E94C111882371F0409A8FEF8093F0
:10073000100110923A0110923B0110923C0110926C
:100740003D0180E0089581E0089580E090E060E060
:1007500040E050E00E94FF104098809196029091F6
:100760009702A0919802B091990280933A019093D8
:100770003B01A0933C01B0933D010895EF92FF929D
:100780000F931F93DF93CF9300D000D000D0CDB74D
:10079000DEB77C010E943D0DDC01F7018381082F4B
:1007A00010E01695102F0027179507952281822FAC
:1007B00090E0082B192BAE014F5F5F4F86E0FA01E6
:1007C00011928A95E9F7F70181818930E9F08A3041
:1007D00030F4833069F0853009F07BC00FC080327F
:1007E00009F463C08332E1F08C3109F072C05FC05C
:1007F000822F0E9493006DC00E94C707C8010E940B
:10080000420D0097C9F765C0109709F462C01296AF
:100810001C930E931197F701848113968C9359C002
:10082000F7018581882311F420E001C020E8C80188
:1008300068E070E00E94021269832A83C801877011
:10084000907083309105F1F0843091054CF4813043
:100850009105A1F0823091059CF4892B69F01CC0B0
:100860008530910599F08530910574F086309105B9
:1008700079F0079789F40EC021600DC022600BC08B
:10088000246009C0286007C0216105C0226103C03F
:10089000246101C028612A8380E260E042E49E0175
:1008A0002F5F3F4F0E94A00414C00E946901F7010E
:1008B0008281882371F48EE6898382E08A8381E0D5
:1008C0008B831C828FEF6CE1AE014F5F5F4F0E9404
:1008D000901180919D02882381F0F701208130E002
:1008E0002F7730708091100190E02817390729F494
:1008F00080919D02815080939D0226960FB6F894B8
:10090000DEBF0FBECDBFCF91DF911F910F91FF9042
:10091000EF900895FC018181893159F02091C20145
:100920003091C3012115310551F0CF01F90109952D
:10093000089584818093C90181E08093C80108955E
:10094000CF93DF93582FE9019091C00182E1989FE6
:10095000F0011124EC5AFE4F652B608342834F70E7
:10096000DF01139603C089918D9341504423D9F739
:10097000503211F481E001C083E081838091C00195
:100980008F5F8093C0018091C001863010F010927B
:10099000C0019091C0018091C101981759F48091D4
:1009A000C1018F5F8093C1018091C101863010F039
:1009B0001092C101DF91CF910895DF93CF93CDB70E
:1009C000DEB72F970FB6F894DEBF0FBECDBF0E94E3
:1009D0006700833061F0843061F09E012F5F3F4FEC
:1009E000823081F4198280E660E041E80FC081E046
:1009F00001C082E0898380E660E041E69E012F5FCE
:100A00003F4F04C0198280E660E041E60E94A004E6
:100A10002F960FB6F894DEBF0FBECDBFCF91DF91FA
:100A20000895DF92EF92FF920F931F93CF93DF937E
:100A3000EC01062F7A012115310519F42FEF3FEF54
:100A400043C0C9010E94AA0F9093C3018093C201C1
:100A5000D093C501C093C4011092C8018EEF9FEFDF
:100A60009093C7018093C60110E084E0D82E002344
:100A700029F080E0602FA7010E949011D0929D0282
:100A800002C00E946A008091C801882321F48091ED
:100A90009D028823B1F70E94A20F811110E080917E
:100AA000C801882319F41F5F183008F38091C20130
:100AB0009091C3010E94AA0F1092C3011092C2012B
:100AC0002091C6013091C701C901DF91CF911F91DB
:100AD0000F91FF90EF90DF900895EF92FF920F93A8
:100AE0001F93DF93CF9300D000D000D0CDB7DEB7F7
:100AF0008C017E010894E11CF11C86E0F701119243
:100B00008A95E9F7F8018385807F8387C7010E9472
:100B10008411C8016EE0A70120E136E00E941105B2
:100B200026960FB6F894DEBF0FBECDBFCF91DF91F2
:100B30001F910F91FF90EF900895EF92FF920F9306
:100B40001F93DF93CF9300D000D000D0CDB7DEB796
:100B50008C01FC01618172817E010894E11CF11C11
:100B6000C7010E948411F801648160956078458115
:100B70005681C7010E946D1180E063E0A7010E94C9
:100B80009011F8016481607845815681C7010E9407
:100B90006D1180E063E0A7010E94901126960FB6C8
:100BA000F894DEBF0FBECDBFCF91DF911F910F91A3
:100BB000FF90EF900895EF92FF920F931F93DF93B2
:100BC000CF9300D000D000D0CDB7DEB78C01FC01B0
:100BD000618172817E010894E11CF11CC7010E94B1
:100BE0008411F80145815681C70164810E946D110D
:100BF00080E063E0A7010E94901188E0F8018187FE
:100C000083858F77838726960FB6F894DEBF0FBE55
:100C1000CDBFCF91DF911F910F91FF90EF9008957D
:100C2000EF92FF920F931F93CF93DF93FC01C0913C
:100C3000C401D091C501209721F481E08093C801BF
:100C4000BCC08381282F30E03695322F222737957C
:100C50002795828190E0282B392B8181893081F082
:100C60008A3020F4873008F4A8C011C08D3009F410
:100C700065C08D3008F4A1C0803108F09EC007C067
:100C80003A83298384818B838B85846094C095818A
:100C9000668177818F3011F0883019F48B858260FE
:100CA0008AC03A832983392F330F330F20E044273A
:100CB00037FD4095542F8D819E81AF81B88580701E
:100CC0009070282B392B4A2B5B2B862F90E08F7747
:100CD0009070A3E0880F991FAA95E1F7AA2797FDC6
:100CE000A095BA2F282B392B4A2B5B2B872F90E00E
:100CF0008077907064E0959587956A95E1F7AA27CB
:100D000097FDA095BA2F282B392B4A2B5B2B2D83CF
:100D10003E834F835887858190E080749070880F60
:100D2000991F2481282B2C832B85822F81608B8710
:100D3000878180FD51C023602B874EC0848190E065
:100D4000A0E0B0E08F779070A070B0708C01FF24AD
:100D5000EE24268130E040E050E07EE1220F331F98
:100D6000441F551F7A95D1F78D819E81AF81B8853B
:100D7000A070B070282B392B4A2B5B2B2E293F29D2
:100D8000402B512B858190E0A0E0B0E08F779070F0
:100D9000A070B07067E1880F991FAA1FBB1F6A95EA
:100DA000D1F7282B392B4A2B5B2B2D833E834F8386
:100DB00058878B8588608B870FC02091C201309146
:100DC000C3012115310521F0CF01F90109950FC0AB
:100DD000CF010E94BE030BC08B858F708F3039F41A
:100DE00081E08093C8011092C7011092C601DF9183
:100DF000CF911F910F91FF90EF900895EF92FF9286
:100E00000F931F93CF93DF93162FE42E052F0E948D
:100E10007202812F0E943E02F82E1F702E2D302F5D
:100E2000C901EC0104C089910E943E02F8269E018E
:100E30002E192117C0F38F2D0E943E02DF91CF9112
:100E40001F910F91FF90EF900895DF93CF93CDB74F
:100E5000DEB72F970FB6F894DEBF0FBECDBF6D89FA
:100E6000762F7F70CE014696DC0120E030E0AE01A7
:100E70004F5F5F4F08C0FA01E20FF31F8C91808330
:100E80002F5F3F4F12967217B1F78C890E94FE06B2
:100E90002F960FB6F894DEBF0FBECDBFCF91DF9176
:100EA00008951F93CF93DF93182FEB018B810E943E
:100EB000F811982F8B3120F08D3120F08E3721F0F2
:100EC000A0E003C0A2E001C0A4E08985883009F059
:100ED000A860EC816E2F6F779B51923078F461118E
:100EE0006D5F862F90E08170907074E0880F991F7D
:100EF0007A95E1F766956F70682B02C061116F5F9C
:100F00002D813E814F815885C90181709070892B58
:100F100011F470E001C070E1E0786E2B8DB79EB7E0
:100F20000A970FB6F8949EBF0FBE8DBFEDB7FEB700
:100F300031961066CDB7DEB7198384EE8183A28324
:100F4000138264831582DA01C9018E719070A070DA
:100F5000B070B695A79597958795782B768317826D
:100F600015E056954795379527951A95D1F720871F
:100F700011860E9425078DB79EB70A960FB6F89482
:100F80009EBF0FBE8DBFDF91CF911F9108950F932C
:100F90001F93DF93CF93CDB7DEB72F970FB6F8949B
:100FA000DEBF0FBECDBF8C010097F1F080E48983D6
:100FB000F80121813281832F992787FD9A95982FF7
:100FC0008A832436310514F0906C9A83F80181816C
:100FD0008B838081806663EEAE014F5F5F4F0E941E
:100FE000FE0687E0F80182872F960FB6F894DEBFE1
:100FF0000FBECDBFCF91DF911F910F910895BF928A
:10100000CF92DF92EF92FF920F931F93DF93CF93D4
:1010100000D000D000D0CDB7DEB77C016B010097C7
:1010200009F46BC06115710509F467C0DC01119604
:101030008D919C91129719962C918617970719F408
:10104000283059F458C0283019F487E0F701818717
:10105000D7011296DC92CE921197C6010E94420DE2
:10106000FC01009719F18E159F0501F18181928194
:10107000D70112969C938E931197838113968C932C
:101080001397848114968C93149725813681478118
:10109000508515962D933D934D935C931897CF01F2
:1010A0000E94C70788E0F701828725C0F6E0BF2EBF
:1010B0008E010F5F1F4FD801EB2D1D92EA95E9F7C6
:1010C000D7011B968C911B97807F1B968C93C80130
:1010D000B6010E948411C70161E0A80120E136E059
:1010E0000E94110597FF03C0F701B28606C088E091
:1010F000D7011A968C9381E001C080E026960FB646
:10110000F894DEBF0FBECDBFCF91DF911F910F913D
:10111000FF90EF90DF90CF90BF900895DF92EF9215
:10112000FF920F931F93DF93CF9300D000D000D096
:10113000CDB7DEB7AC012FEF8F3F920769F186E0A4
:1011400080939A0280913E01882329F410925301E2
:10115000109252014EC420915201213168F4E22FC5
:10116000F0E0EF5BFE4F4083809153018427809332
:1011700053012F5F2093520120915201223008F435
:1011800038C430E08091410190E08F7090700296F9
:101190002817390709F02DC40E94B602882319F0D8
:1011A00086E080939A0280919A028823E1F011E010
:1011B00015C0812F60E00E94620DFC01009751F084
:1011C0008185883039F4838587FF04C0CF010E9470
:1011D000DB050FC41F5F1F3109F40BC40E940D0E05
:1011E00004973CF706C440915201242F30E08091CF
:1011F000410190E08F70907002962817390709F02E
:1012000051C380915301882309F04CC30E94B40F4D
:10121000D0903E018F3F81F400D000D0EDB7FEB7F3
:10122000319630E6D32AADB7BEB71196DC9281E68F
:10123000818381E890E048C3409A8D2D61E00E944F
:10124000A70D8C01009709F4FCC2FC018185863052
:1012500081F400D000D0EDB7FEB7319620E6D22A57
:10126000ADB7BEB71196DC9281E6818381E890E04C
:10127000F7C2823018F482E0F80181879091410131
:10128000892F82958F70853009F4F2C0863030F452
:10129000823071F0843009F0D4C275C0893009F40D
:1012A00049C28E3009F413C1883009F0CAC209C19D
:1012B000903221F4D8011A961C92DAC28091420130
:1012C000843259F1853220F4813209F0B2C207C06C
:1012D000803809F445C0813809F0ABC249C0EDB788
:1012E000FEB738970FB6F894FEBF0FBEEDBF31962C
:1012F00020E6D22AADB7BEB71196DC9283E6818391
:1013000081E290E09383828386E390E095838483F7
:1013100081E090E097838683C4C10E946700823099
:1013200011F421E009C0882311F422E005C08430C3
:1013300011F428E001C020E000D000D000D0EDB7CB
:10134000FEB7319630E6D32AADB7BEB71196DC9220
:1013500082E6818382E290E093838283248381C04A
:101360000E946700882341F080E060E240E0ACC06A
:101370000E946700833019F40E94DD0479C280E086
:1013800060E243E0A1C080914201E82EFF24EE0C10
:10139000FF1CEE0CFF1C8091430180FF04C0E2E0C3
:1013A000F0E0EE0EFF1EE1FC02C010E001C010E113
:1013B00081E491E0B7010E94841180E090E069E14E
:1013C00041E451E02AE834E00E9411058091C9010E
:1013D000823551F083351CF4873459F408C08736C0
:1013E00039F0823731F401C01068116002C0106812
:1013F0001260B7016F5F7F4F81E491E00E9484111A
:1014000080E090E069E141E451E02AE834E00E94A4
:1014100011058091C901823551F083351CF4873460
:1014200059F408C0873639F0823731F401C01068AA
:10143000146002C01068186000D000D000D0EDB772
:10144000FEB7319620E6D22AADB7BEB71196DC9230
:1014500082E48183F694E794F694E794F382E2823F
:10146000148315820E942507EDB7FEB736961EC17C
:101470006091420170E093E0660F771F9A95E1F763
:101480000091430110E0C80187709070682B792BA0
:1014900081E090E0682779277E010894E11CF11C27
:1014A000C7010E9484111B8283E0169507958A95D7
:1014B000E1F701700C8380E066E0A7010E949011C3
:1014C000D7C180E060E242E00E94A611D1C19091B4
:1014D000430180E020914401E22EFF24E82AF92A0A
:1014E0002FEF3FE3E222F322809142018331A8F4FF
:1014F000813108F0E1C0883009F482C0893030F4CD
:101500008823D9F0873009F094C160C0893009F48C
:101510009DC0803109F08DC1F7C0803209F415C13A
:10152000813220F4833109F084C1F3C0813209F49F
:101530003FC1823209F07DC158C1D80111968D9109
:101540009C911297E816F906A1F119968C911997BA
:10155000883019F487E019968C93C7010E94420DD8
:10156000FC010097E9F080179107D1F08181928109
:10157000D80112969C938E931197838113968C9326
:101580001397848114968C9385819681A781B08569
:10159000F80185839683A783B08787E0818704C09D
:1015A000C801B7010E946D058D2DB8010E94510739
:1015B0005FC18D2DB8010E945107D80111966D9120
:1015C0007C911297C8010E946D0552C1EDB7FEB71C
:1015D00038970FB6F894FEBF0FBEEDBF319620E6E8
:1015E000D22AADB7BEB71196DC9283EE818380E537
:1015F00090E093838283158214821782168251C0F1
:101600002DB73EB72A5030400FB6F8943EBF0FBEFC
:101610002DBFEDB7FEB7319630E6D32AADB7BEB7D2
:101620001196DC9284EE818381E590E0938382833E
:1016300015821482178216828FE090E0918780874E
:101640000E942507EDB7FEB73A9630C0D80115962F
:101650004D915D916D917C911897EDB7FEB73897DC
:101660000FB6F894FEBF0FBEEDBF319620E6D22A2A
:10167000ADB7BEB71196DC9223EE218322E530E0B0
:1016800033832283BDE07695679557954795BA9544
:10169000D1F744831582BB27A72F962F852F8683EA
:1016A00017820E942507EDB7FEB738960FB6F8945B
:1016B000FEBF0FBEEDBFDCC0C801B7010E94FF072F
:1016C000882309F4D5C040914501842F90E09C0106
:1016D0002071307054E0359527955A95E1F78F7059
:1016E0009070880F991F282B822F8150823028F408
:1016F0004078D80114964C931DC021112350407896
:10170000242BF801248391C0809145018F78809328
:101710004501C801B7010E94FF07882309F4A8C04A
:1017200090914501892F8F77813041F49078D801CD
:1017300014969C93C8010E949D059AC08111815006
:101740009078892BF801848370C0C801B7010E948A
:10175000FF07882309F48CC080914501D8011596B4
:101760002D913D914D915C91189784FF07C02160A8
:10177000F801258336834783508708C02E7FD80120
:1017800015962D933D934D935C9318978091450149
:1017900090E08F709070880F991FAA2797FDA095F1
:1017A000BA2FF8012581368147815085217E35C0C9
:1017B000C801B7010E94FF07882309F459C080912E
:1017C000450190E08F709070B5E0880F991FBA9531
:1017D000E1F7AA2797FDA095BA2FF8012581368158
:1017E000478150852F713E7F18C0C801B7010E9404
:1017F000FF078823E9F18091450190E08F70907098
:10180000982F8827990FAA2797FDA095BA2FF8013E
:101810002581368147815085317E822B932BA42BE5
:10182000B52B85839683A783B087C8010E94DB050B
:101830001FC000D000D0EDB7FEB7319620E6D22A07
:1018400007C000D000D0EDB7FEB73196B0E6DB2A76
:10185000ADB7BEB71196DC9281E6818382E890E055
:10186000938382830E9425070F900F900F900F9013
:10187000409880913E0160E00E94620D8C010097CB
:1018800059F1FC018385806883870E940D0E0397C0
:101890001CF1D80119968C918830F1F4C8010E948E
:1018A000DB051AC04423C1F000D000D0EDB7FEB76D
:1018B000319680913E018066ADB7BEB711968C938C
:1018C00081E6818380E890E0938382830E942507EC
:1018D0000F900F900F900F901092530110925201A1
:1018E00011E00CE0812F60E00E94620DFC01009786
:1018F00069F08285882351F0893031F4DF01202F8F
:101900001D922A95E9F702C0818712861F5F103267
:1019100049F70E94B602882309F06BC09091C0017C
:101920008091C101981729F14091C10182E1489F3E
:10193000800111240C5A1E4FA8014D5F5F4FD80142
:101940008C9112966C910E94FE06F8018181815063
:101950008183882309F04AC08091C1018F5F809301
:10196000C1018091C101863008F440C01092C101CC
:101970003DC080914001882361F480913F018F5FD9
:1019800080933F01803228F010923F0181E08093E4
:10199000400180913F01882351F060E00E94620D78
:1019A000892B29F480913F0180933E011CC08091D6
:1019B0003E010E94B50DFC01009751F0808180939B
:1019C0003E018185863031F4CF010E94C70702C0F5
:1019D00010923E01809140018F5F80934001809181
:1019E0003E01882319F080640E94720286E0809391
:1019F0009A0226960FB6F894DEBF0FBECDBFCF91E8
:101A0000DF911F910F91FF90EF90DF900895482F85
:101A100050E020E030E08091CA01882311F421E0F9
:101A200030E02417350731F120E030E08091D60115
:101A3000882311F421E030E024173507D9F020E0A5
:101A400030E08091E201882311F421E030E0241796
:101A5000350781F090E020E030E08091EE018823AE
:101A600011F421E030E02417350709F491E081E01A
:101A7000982701C090E0892F08958091FA019091F4
:101A8000FB0108959C01EAECF1E00CC082858823FB
:101A900009F48185883029F4818192818217930726
:101AA00039F03C9681E0EA3FF80781F7E0E0F0E0AA
:101AB000CF01089580E3EAECF1E0DF011D928A9501
:101AC000E9F70895CF93DF93382F81508F31C8F510
:101AD000CAECD1E004C088818317A9F12C9681E07B
:101AE000CA3FD807C1F7662361F120E0E09725C01F
:101AF0008881882301F5388382E0898700D000D06F
:101B000000D0EDB7FEB7319688E690E0ADB7BEB72E
:101B100012969C938E93119732831382248315829D
:101B20000E9429128DB79EB706960FB6F8949EBFF5
:101B30000FBE8DBF08C02C962F5F91E0CA3FD9071A
:101B4000B8F2C0E0D0E0CE01DF91CF9108958823B4
:101B500019F420E030E003C00E94620D9C01309334
:101B6000FB012093FA01C90108950F931F93182FC9
:101B7000882311F401E005C0803210F00FE101C0AC
:101B8000082F1F5F103208F011E0812F60E00E94E3
:101B9000620D9C01101711F0009799F3C9011F9174
:101BA0000F91089580E090E008958FEF9FEF0895E2
:101BB000089580E0089580E090E008958FEF9FEF12
:101BC0000895DC019091840289E0989FF00111242E
:101BD000EA5FFD4F90E08D9181939F5F9930D9F737
:101BE000809184028F5F809384028091840286308A
:101BF00010F01092840208951092900210928902BF
:101C0000109288020895909184028091850220E0CC
:101C1000981709F421E0822F08958FB7F8949091D6
:101C2000840220918502492F50E0421B51098FBF49
:101C300057FF02C04A5F5F4F25E030E0241B350BA1
:101C4000C90108951F93AC011FB7F8942091840235
:101C50008091850230E090E001972817390741F024
:101C600080918402853039F480918502882319F4AB
:101C70001FBF80E005C0CA010E94E10D1FBF81E0C7
:101C80001F910895DC01EDEFF1E08D91819382E0E9
:101C9000E630F807D1F708959C01009739F14FB766
:101CA000F8949091860280918702981721F44FBF93
:101CB00020E030E01BC09091870289E0989FF001FE
:101CC0001124E45CFD4FD90190E081918D939F5FD9
:101CD0009930D9F7809187028F5F80938702809136
:101CE0008702883010F0109287024FBFC901089513
:101CF0001F93182F87FF86C08091860290E001967F
:101D00009C0143E0220F331F4A95E1F7280F391F4A
:101D1000245C3D4F80918A0290918B028217930739
:101D2000E1F4809186028F5F809386028091860223
:101D3000883010F01092860290918602809187027E
:101D4000981759F4809187028F5F80938702809162
:101D50008702883010F01092870210928B02109246
:101D60008A0210928902109288028091100118173D
:101D700021F481E08093900277C010929002412F6D
:101D800050E04F775070682F70E04617570729F0E2
:101D90001F3F19F08F3F09F067C08091860229E04C
:101DA000829FC0011124845C9D4F90938B0280938D
:101DB0008A024617570709F057C090918402809114
:101DC0008502981721F48DEF91E00E94E10D80913A
:101DD000850229E0829FC00111248A5F9D4F909364
:101DE000890280938802809185028F5F80938502AB
:101DF00080918502863010F01092850289E08093F0
:101E0000FC0132C020919002213029F0213060F194
:101E1000263050F515C082E080939002103419F4FA
:101E20001092910221C0113419F4209391021CC028
:101E3000123419F0133491F483E08093910214C0AA
:101E4000E22FF0E08091910290E002968E179F07BA
:101E500044F0E657FD4F8081181719F01092900258
:101E600003C02F5F209390020E946700883021F109
:101E700080919002882329F010939B0210929C027B
:101E800021C0E0918802F09189023097A9F08191F8
:101E900080939B0210929C02F0938902E093880247
:101EA0008091FC0181508093FC01882359F41092A9
:101EB00089021092880206C08FEF9FEF90939C02D8
:101EC00080939B02E0918A02F0918B02309749F057
:101ED00082E0E438F80728F41193F0938B02E09342
:101EE0008A021F9108958FEF9FEF90939C02809339
:101EF0009B020E945A01262F2F7720938F02F7E032
:101F00009695879577956795FA95D1F7262F2F7730
:101F100020938E02E7E09695879577956795EA95E9
:101F2000D1F7262F2F7720938D0257E0969587952E
:101F3000779567955A95D1F76F7760938C020E94D9
:101F40001A03089580919402882319F01092940244
:101F500081E0089520919202309193029093930230
:101F600080939202C90108958091100108950F9302
:101F70001F93DF93CF93CDB7DEB729970FB6F894B1
:101F8000DEBF0FBECDBFDA01A89580911001806839
:101F900089836A83FE0133969E01275F3F4F109726
:101FA00021F08D918F77808301C010823196E217E6
:101FB000F307A9F78E010F5F1F4FC8010E94471159
:101FC0008987C8010E94220E29960FB6F894DEBFB9
:101FD0000FBECDBFCF91DF911F910F9108952F922A
:101FE0003F924F925F926F927F928F929F92AF92A9
:101FF000BF92CF92DF92EF92FF920F931F93DF93E6
:10200000CF93CDB7DEB729970FB6F894DEBF0FBEDA
:10201000CDBF809110018F3F09F06FC00E945A011F
:102020009B01AC0139014A0177E09594879477943C
:1020300067947A95D1F78FE790E0A0E0B0E068224E
:1020400079228A229B2259016A016EE0D594C794B5
:10205000B794A7946A95D1F7A822B922CA22DB22A5
:1020600079018A0195E115950795F794E7949A957A
:10207000D1F787E090E0A0E0B0E0E822F9220A235F
:102080001B238FE7282E312C412C512C2222332266
:102090004422552234C0A8958A81843081F5CE012E
:1020A00001960E945E11882351F18E8190E0A0E09C
:1020B000B0E0281639064A065B0609F58D8190E0E6
:1020C000A0E0B0E0681679068A069B06C1F48C8110
:1020D00090E0A0E0B0E0A816B906CA06DB0679F4E5
:1020E0008B8190E0A0E0B0E0E816F9060A071B0734
:1020F00031F489818F778093100181E007C0CE0190
:1021000001960E944C0E892B31F680E029960FB67D
:10211000F894DEBF0FBECDBFCF91DF911F910F911D
:10212000FF90EF90DF90CF90BF90AF909F908F90F7
:102130007F906F905F904F903F902F900895DF9227
:10214000EF92FF920F931F93DF93CF93CDB7DEB73C
:1021500029970FB6F894DEBF0FBECDBF8091100156
:102160008F3F89F50E94EF0F8823D9F180911001EC
:102170000E94A50336C0C8010E945E11882361F148
:10218000298130E02F7730708091100190E028177E
:10219000390711F40E946B038A81863019F4D092BA
:1021A00094021AC08091920290919302892B21F49B
:1021B000F0929302E0929202E0919202F0919302E7
:1021C000C801099509C08E010F5F1F4FEEEBEE2E7F
:1021D000E3E0FE2EDD24D394C8010E944C0E892B2F
:1021E00051F629960FB6F894DEBF0FBECDBFCF9142
:1021F000DF911F910F91FF90EF90DF9008950F9363
:102200001F93DF93CF93CDB7DEB729970FB6F8941E
:10221000DEBF0FBECDBF209110012068298323E0CF
:102220002A83282F2F772B83880F892F881F990BBC
:1022300091958F778C83862F8F778D83852F8695C9
:1022400086958E8367FF02C080648E83CA01F3E0A7
:1022500096958795FA95E1F78F778F83842F8295EE
:10226000807788878E010F5F1F4FC8010E9447113A
:102270008987C8010E94420E29960FB6F894DEBFE6
:102280000FBECDBFCF91DF911F910F910895FC013B
:1022900020E090E037E08191982780E097FF03C02D
:1022A000990F932701C0990F8F5F8830B9F72F5F7F
:1022B000283089F797FD9095892F08950F931F93E4
:1022C0008C010E94471120E0F8019085891709F4DC
:1022D00021E0822F1F910F910895FC01862F8F77A7
:1022E0008283852F8695869566956074862B838379
:1022F000CA0123E0969587952A95E1F78F77848325
:102300004295407745830895FC01862F8F7780831F
:10231000660F672F661F770B71956F77618308953E
:102320000F931F93CF93DF93082F162FEA0102C05C
:102330000E946A00802F612FAE010E94B70F882390
:10234000B9F3DF91CF911F910F910895DF93CF9350
:1023500000D000D000D0CDB7DEB7FE01319696E0B8
:10236000DF011D929A95E9F74983AF010E94901110
:1023700026960FB6F894DEBF0FBECDBFCF91DF918A
:1023800008959B01AC018091960290919702A091D3
:102390009802B091990282179307A407B50798F0A5
:1023A0008091960290919702A0919802B091990223
:1023B00060E0821B930BA40BB50B80509041A040B2
:1023C000B040A0F412C08091960290919702A09123
:1023D0009802B091990260E0281B390B4A0B5B0B05
:1023E0002050304F4F4F5F4F08F061E0862F089527
:1023F000E82FF0E0EF70F070E158FF4FE4918E2F7E
:1024000090E0089597FB092E07260AD077FD04D0A7
:102410000CD006D000201AF4709561957F4F089576
:10242000F6F7909581959F4F0895AA1BBB1B51E12C
:1024300007C0AA1FBB1FA617B70710F0A61BB70B34
:10244000881F991F5A95A9F780959095BC01CD01D9
:102450000895A0E0B0E0EFE2F2E10C94DC14FE019C
:10246000359661917191A091A002B091A10213964D
:102470008C911397886013968C938091A002909111
:10248000A102AF010E944F12E091A002F091A102BF
:102490002381277F23832096E2E00C94F814ABE09D
:1024A000B0E0E5E5F2E10C94CC143C012B015A01BB
:1024B000FC0117821682838181FD03C06FEF7FEFDD
:1024C000C6C19AE0892E1E010894211C311CF3011B
:1024D0002381F20123FD859123FF81912F01882320
:1024E00009F4B2C1853239F423FD859123FF81912E
:1024F0002F01853229F490E0B3010E944214E7CF06
:10250000982FFF24EE249924FFE1FF15D0F09B3291
:1025100069F09C3228F4903259F0933291F40EC055
:102520009D3249F0903369F441E024C052E0F52A2D
:1025300084E0F82A28C098E0F92A25C0E0E1FE2AC4
:1025400022C0F7FC29C0892F80538A3070F4F6FE30
:1025500005C0989C902C1124980E15C0E89CE02C86
:102560001124E80EF0E2FF2A0EC09E3229F4F6FC98
:102570006BC140E4F42A07C09C3619F450E8F52AF0
:1025800002C0983649F4F20123FD959123FF919101
:102590002F01992309F0B8CF892F8554833018F083
:1025A0008052833038F444E050E0A40EB51E5FE35F
:1025B00059830FC0933631F0933779F0933509F092
:1025C00056C020C0F5018081898342E050E0A40E0E
:1025D000B51E610101E010E012C0F501C080D1809C
:1025E000F6FC03C06FEF7FEF02C0692D70E042E0A0
:1025F00050E0A40EB51EC6010E9437148C015FE79F
:10260000F52214C0F501C080D180F6FC03C06FEF45
:102610007FEF02C0692D70E042E050E0A40EB51ECD
:10262000C6010E942C148C0150E8F52AF3FE07C065
:102630001AC080E290E0B3010E944214EA948E2D09
:1026400090E008171907A8F30EC0F601F7FC859172
:10265000F7FE81916F0190E0B3010E944214E110F6
:10266000EA94015010400115110579F7EAC094363B
:1026700011F0993669F5F7FE08C0F5012081318126
:102680004281538184E090E00AC0F501808191810C
:102690009C01442737FD4095542F82E090E0A80E1E
:1026A000B91E9FE6F92257FF09C050954095309515
:1026B00021953F4F4F4F5F4FE0E8FE2ACA01B90115
:1026C000A1012AE030E00E946E14D82ED21840C03A
:1026D000953729F41F2D1F7E2AE030E01DC01F2DE5
:1026E000197F9F3661F0903720F4983509F0ACC01F
:1026F0000FC0903739F0983709F0A6C004C028E021
:1027000030E00AC0106114FD146020E130E004C024
:1027100014FD166020E132E017FF08C0F50160816A
:1027200071818281938144E050E008C0F50180818D
:102730009181BC0180E090E042E050E0A40EB51E23
:10274000A1010E946E14D82ED2188FE7F82EF12224
:10275000F6FE0BC05EEFF522D91438F4F4FE07C084
:10276000F2FC05C08FEEF82202C01D2D01C0192D0C
:10277000F4FE0DC0FE01ED0DF11D8081803319F4D2
:1027800099EEF92208C01F5FF2FE05C003C08F2D2D
:10279000867809F01F5F0F2DF3FC14C0F0FE0FC008
:1027A0001E1510F09D2C0BC09D2C9E0C911A1E2DF9
:1027B00006C080E290E0B3010E9442141F5F1E1524
:1027C000C0F304C01E1510F4E11A01C0EE2404FF8A
:1027D0000FC080E390E0B3010E94421402FF1DC0CD
:1027E00001FD03C088E790E00EC088E590E00BC0D3
:1027F000802F867891F001FF02C08BE201C080E259
:10280000F7FC8DE290E0B3010E94421406C080E321
:1028100090E0B3010E9442149A94D914C0F3DA9460
:10282000F101ED0DF11D808190E0B3010E94421491
:10283000DD20A9F706C080E290E0B3010E944214B7
:10284000EA94EE20C1F743CEF30166817781CB0194
:102850002B96E2E10C94E814FC0105906150704065
:102860000110D8F7809590958E0F9F1F0895FC0159
:102870006150704001900110D8F7809590958E0FAF
:102880009F1F08950F931F93CF93DF938C01EB014C
:102890008B8181FF1BC082FF0DC02E813F818C8107
:1028A0009D812817390764F4E881F9810193F98340
:1028B000E88306C0E885F985802F0995892B31F4D6
:1028C0008E819F8101969F838E8302C00FEF1FEF41
:1028D000C801DF91CF911F910F910895FA01AA27A6
:1028E000283051F1203181F1E8946F936E7F6E5F53
:1028F0007F4F8F4F9F4FAF4FB1E03ED0B4E03CD001
:10290000670F781F891F9A1FA11D680F791F8A1FE3
:10291000911DA11D6A0F711D811D911DA11D20D04A
:1029200009F468943F912AE0269F11243019305D04
:102930003193DEF6CF010895462F4770405D4193F5
:10294000B3E00FD0C9F7F6CF462F4F70405D4A3342
:1029500018F0495D31FD4052419302D0A9F7EACF0A
:10296000B4E0A6959795879577956795BA95C9F739
:1029700000976105710508959B01AC010A2E06942C
:102980005795479537952795BA95C9F7620F731FE5
:10299000841F951FA01D08952F923F924F925F9222
:1029A0006F927F928F929F92AF92BF92CF92DF925F
:1029B000EF92FF920F931F93CF93DF93CDB7DEB7C4
:1029C000CA1BDB0B0FB6F894DEBF0FBECDBF099458
:1029D0002A88398848885F846E847D848C849B84AF
:1029E000AA84B984C884DF80EE80FD800C811B81BD
:1029F000AA81B981CE0FD11D0FB6F894DEBF0FBEEC
:0A2A0000CDBFED010895F894FFCF5B
:102A0A0000808000800000808000008000808000BC
:022A1A00FF00BB
:00000001FF
